:1000000055AA55AA0200000036700000000000004A
:100010006622000000000000100000000000000048
:1000200000000000000000000F00000074650000E8
:10003000000800000000000000000000047627F91E
:100040000C4F48B45C190000F3B0B74BA3E6FFFFB8
:1000500000021000E10000008B510000A10100002F
:10006000ED010000390200008502000000000000E0
:100070000000000000000000000000008F510000A0
:100080009751000000000000D10200009F510000C5
:10009000A7510000B5510000BD510000CB51000038
:1000A000D9510000E7510000EF510000FD51000060
:1000B0004B520000DF0200000B5200001352000000
:1000C00000000000235200004D5200004F5200007B
:1000D0005D5200005F520000615200003B52000080
:1000E000435200002B5200003352000063520000C4
:1000F00065520000735200001B5200000000000017
:1001000000000000000000000000000000000000EF
:100110006622000001000140000000000000000015
:1001200000000000000000000000000000000000CF
:1001300000F002F800F03AF80AA090E8000C8244BF
:100140008344AAF10107DA4501D100F02FF8AFF29C
:10015000090EBAE80F0013F0010F18BFFB1A43F0A5
:10016000010318470062000030620000103A24BF0B
:1001700078C878C1FAD8520724BF30C830C144BF0C
:1001800004680C607047000000230024002500264E
:10019000103A28BF78C1FBD8520728BF30C148BFEA
:1001A0000B6070471FB51FBD10B510BDDFF80CD038
:1001B000FFF7F8FF05F019F905F032FD0002100015
:1001C00003B4FFF7F1FF03BC05F032FD40BA7047FE
:1001D000C0BA704772B6784600F10A004DF8080CB4
:1001E00062B630BF00BF704740BA7047C0BA7047B0
:1001F00011484FF00F0100F8011B4FF0010100F80A
:10020000011B4FF0020100F8011B4FF0000100F844
:10021000011B00F8011B00F8011B00F8011B00F88E
:10022000011B1EF0040F0CBFEFF30880EFF30980F1
:100230004FF0020103F01ABF0002002011484FF0F6
:100240000F0100F8011B4FF0010100F8011B4FF0F6
:10025000030100F8011B4FF0000100F8011B00F83A
:10026000011B00F8011B00F8011B00F8011B1EF028
:10027000040F0CBFEFF30880EFF309804FF0030188
:1002800003F0F4BE0002002011484FF00F0100F807
:10029000011B4FF0010100F8011B4FF0040100F8B1
:1002A000011B4FF0000100F8011B00F8011B00F8D2
:1002B000011B00F8011B00F8011B1EF0040F0CBF0E
:1002C000EFF30880EFF309804FF0040103F0CEBE96
:1002D0000002002011484FF00F0100F8011B4FF001
:1002E000010100F8011B4FF0050100F8011B4FF060
:1002F000000100F8011B00F8011B00F8011B00F8C9
:10030000011B00F8011B1EF0040F0CBFEFF3088067
:10031000EFF309804FF0050103F0A8BE00020020B2
:1003200000B504F051FF5DF804EB00F02FB81EF0AB
:10033000040F0CBFEFF30880EFF309804FF00001CA
:1003400003F094BE0A484FF0FF0101704FF0000027
:1003500080F311884FF0000080F3098805484FF0C2
:100360000201017062B604484FF08051016070478D
:1003700022ED00E00B03100004ED00E002484FF016
:10038000805101607047000004ED00E04FF0200054
:1003900080F31188EFF3098098B112480068124980
:1003A0000968884217D0EFF309800E49096820E9EF
:1003B000F00F886000B50B48006805F0EAF85DF8BA
:1003C00004EB084808490A68026000688168B1E8DF
:1003D000F00F81F309884EF0040E4FF0000080F317
:1003E000118870470C03100010031000EFF3118008
:1003F0004FF0200181F31188704700004FF000009A
:1004000080F311887047000062B6704772B670477B
:1004100010B5022000F00AFA032000F007FA0420C9
:1004200000F004FA052000F001FA062000F0FEF9C1
:10043000072000F0FBF9082000F0F8F9092000F08F
:10044000F5F90F2000F0F2F94FF00051002001F80B
:100450004A0F8871F022CA710F224A70F949086266
:1004600088620863886008618861C8604861C86103
:100470004862C86248630621022000F0F6F90621AE
:10048000032000F0F2F90621042000F0EEF9062125
:10049000052000F0EAF90621084600F0E6F90621F9
:1004A000072000F0E2F90621082000F0DEF904211F
:1004B000092000F0DAF906210F2000F0D6F9022019
:1004C00000F0C8F9032000F0C5F9042000F0C2F9DB
:1004D000052000F0BFF9062000F0BCF9072000F06D
:1004E000B9F9082000F0B6F9092000F0B3F90220AC
:1004F00000F091F9032000F08EF9042000F08BF950
:10050000052000F088F9062000F085F9072000F0AA
:1005100082F9082000F07FF9BDE81040092000F0C2
:100520007AB94FF00051C98C4FEA90100A06C549BC
:1005300001D5C54A00E0C54AB2FBF0F0086070473B
:100540004FF0005090F84A00000700D0012070479B
:100550007047BF4900200860BA498860C86070478A
:10056000B84AD160642148430A2190FBF1F0B0F50C
:10057000803F06DBA0F57F40FF3890604FF6FF70AC
:1005800002E0002180B2916000F07FB9AD4910B562
:100590008868B0F5803F06DBA0F57F40FF388860B3
:1005A0004FF6FF7003E030B10022C0B28A60BDE8B0
:1005B000104000F06AB9CA68FFF7CBFF12B1BDE87E
:1005C000104010470020FFF7C3FF10BDA0490020D6
:1005D000091D08609B49086148617047994A51614B
:1005E000642148430A2190FBF1F0B0F5803F06DB1F
:1005F000A0F57F40FF3810614FF6FF7002E0002148
:1006000080B2116100F04BB98E4910B50869B0F5A0
:10061000803F06DBA0F57F40FF3808614FF6FF7092
:1006200004E0002806DD002280B20A61BDE8104027
:1006300000F035B94A69FFF7C9FF12B1BDE81040B3
:1006400010470120FFF784FF10BD814900200831C9
:1006500008607C498861C86170477A4910B588692B
:10066000B0F5803F06DBA0F57F40FF3888614FF68C
:10067000FF7003E030B1002280B28A61BDE8104013
:1006800000F017B9CA69FFF7E0FF12B1BDE81040EA
:1006900010470220FFF75CFF10BD6D4900201031AC
:1006A00008606849086248627047664910B5086A80
:1006B000B0F5803F06D3A0F57F40FF3808624FF6C3
:1006C000FF7003E030B1002280B20A62BDE8104042
:1006D00000F0F9B84A6AFFF7E0FF12B1BDE8104038
:1006E00010470420FFF734FF10BD59490020143192
:1006F000086054498862C8627047524AD1621168E2
:1007000048430A21B0FBF1F0B0F5803F06DBA0F5CD
:100710007F40FF3890624FF6FF7002E0002180B208
:10072000916200F0DBB84FF00050B0F85A00454934
:10073000096908447047434910B5886AB0F5803F9D
:1007400006D3A0F57F40FF3888624FF6FF7003E0C4
:1007500030B1002280B28A62BDE8104000F0BEB81D
:10076000CA6AFFF7C2FF12B1BDE81040104705206A
:10077000FFF7EEFE10BD4020C10581F82100704753
:10078000334800211C3001604FF000524FF6FF71DA
:10079000A2F866100121016070472D4900201C312C
:1007A000086070474FF0005090F82110C90606D538
:1007B00010F8211F21F01001017001207047002066
:1007C000704710B504460F2000F044F80F2000F0E9
:1007D00022F81C4844604FF00050C18C090602D535
:1007E0004EF6602101E04AF6C871416518490120C2
:1007F000B8310860091D086010BD10B50F2000F069
:1008000015F84FF00050C06C0E4920F07F40496849
:10081000BDE81040084700F01F0201219140400947
:10082000800000F1E020C0F80011704700F01F02C6
:10083000012191404009800000F1E020C0F88011C2
:100840007047000000021000C0270900D0DD06003C
:100850004009002200F01F02012191404009800060
:1008600000F1E020C0F88012EAE74907090E0028ED
:1008700006DA00F00F0000F1E02080F8141DDFE739
:1008800000F1E02080F80014DAE71A4900220A603B
:100890004FF00052A2F8580001200860D0E7154937
:1008A0000022091D0A60CA06A2F85A000120086049
:1008B000C6E71049002208310A608A06A2F85C00E7
:1008C00001200860BCE70B49002210310A604FF09C
:1008D0000052A2F8600001200860B1E7054900223B
:1008E00014310A604FF00052A2F862000120086043
:1008F000A6E700004009002210B55B4C00202060F4
:100900005A4800F09BFD0120206010BD10B54FF04B
:10091000E0214FF08060C1F88001C1F880025449A5
:10092000A02081F80004FFF7E7FF4FF00051C88CCA
:10093000CA8C00F00300120600EB400001D54D4ABE
:1009400001E04C4A303A12F8203001F8983F02EBAF
:10095000800042784A7082788A70C278CA700279C0
:100960000A7142794A7182798A71C279CA71027AAE
:100970000A72427A4A72827A8A72C07AC87210BD4A
:1009800070B54FF0005400F07F00049D84F88D0096
:1009900084F88E10A4F8942001213748002283B1F6
:1009A000C0F8801194F8913023F0700384F89130EE
:1009B00094F89130702606EA05152B4384F891309F
:1009C00001E0C0F8802114F8923F23F03403237033
:1009D000C0F84422C0F84012D0F89C110129FBD184
:1009E00070BDF0B54FF00054DDE90765DDE905C7DE
:1009F00000F07F0084F88D0084F88E10A4F8942015
:100A000084F88F30A4F896C001211B48002287B1DA
:100A1000C0F8801194F8913023F0700384F891307D
:100A200094F89130702707EA05152B4384F891302C
:100A300001E0C0F8802114F8923F23F034032370C2
:100A4000237843F02003237016B1C0F8481201E068
:100A5000C0F84822C0F84422C0F84012D0F89C11D7
:100A60000129FBD1F0BD000084140022AA820600F7
:100A70001AE000E0785C00000010002237480121F5
:100A800001600021016070473548012101600021AB
:100A90000160704700B54FF0E0230122C3F88021C8
:100AA00003F5C073FFF7F0FFFFF7E8FF2C480838A5
:100AB0000260A02083F88002C3F8002143F8802C54
:100AC00000BD2749083910B1002008607047012097
:100AD000FBE723480121783801600021016070475D
:100AE00010B572B61F490C78002104E01D4A521C53
:100AF000525C4254491CA142F8DB40F6FC0000F075
:100B00009DFC62B6204610BD144901201C390860C6
:100B10007047144820300078124921310978401A72
:100B200000F03F0070474FF00051027881F800223A
:100B3000427881F80122827881F80222C27881F815
:100B40000322027981F80422427981F80522827910
:100B500081F80622C07981F8070270475C84002280
:100B6000940500220004002010B50A2000F05AF875
:100B70000B2000F057F80A2000F05FF80B2000F07F
:100B80005CF805210A2000F063F805210B2000F035
:100B90005FF84FF000507F2100F8351F4170C170A1
:100BA0000021C17101724172817210BD0123834025
:100BB000D8B24FF00053002993F8361001D001430A
:100BC00000E0814383F8361013F8381F0AB101435F
:100BD00000E081431970704701238340D8B24FF081
:100BE0000053002993F83C1006D0014383F83C10D1
:100BF00093F83E10014305E0814383F83C1093F8DD
:100C00003E10814383F83E1013F83D1F22B101438B
:100C100019709978014303E08143197099788143F1
:100C20009970704700F01F02012191404009800037
:100C300000F1E020C0F88011704700F01F02012190
:100C400091404009800000F1E020C0F88012704718
:100C50004907090E002806DA00F00F0000F1E02035
:100C600080F8141D704700F1E02080F800147047F0
:100C70007047FE4BFE4A998A814203D2401AD080C7
:100C8000084601E00021D180DA68FA491047F748A8
:100C900010B500698047F649C88810B1BDE810401A
:100CA000E7E78968002903D0BDE810400120084724
:100CB00010BDEE4810B500698047ED4C4FF00000C4
:100CC000A16819B188470020A06010BDFFF7D0FFD0
:100CD00010BDE749CA780B7952005A43E34B0878B4
:100CE000D2B29B6840F48070C96818470146182248
:100CF000DE4804F09BBE38B5DD4A817913231171BB
:100D00004179D170027901F0070102F01F028DF8DC
:100D100000208DF80110C078032200F01F008DF82C
:100D20000200D248694644681846A04738BDF8B565
:100D30000446007CCD4DC0F34002014662F35F01E2
:100D4000C0F3800241EA8201C0F3C00241EAC2015D
:100D5000C0F3001241EA0211C0F3401241EA42110D
:100D60008DF800108109607C272300F0010241EA20
:100D70000211C0F3400041EA40108DF80100607C90
:100D8000C0F38001C0F3C00241EA0211C0F30012B7
:100D900041EA4211C0F3401241EA8211800941EA5E
:100DA000C0108DF802006E68032269461846B047ED
:100DB000E0792B23C0F38002014662F39F01C0F368
:100DC000C10241EA0211C0F3401041EA80108DF8DF
:100DD0000000607CA17CC00901F0030140EA011021
:100DE0008DF801006E68022269461846B0472D262C
:100DF0002B680122694630469847A17C9DF8000087
:100E0000C1F3800108438DF800006B680122694638
:100E100030469847F8BD10B50446FFF76CFF2046F2
:100E200000F04FF92046BDE8104080E738B53D217D
:100E30008DF800108D49044612204B680122694646
:100E40009847A088FFF715FF38BD10B5044600F09D
:100E50007AF92046BDE81040E8E7F8B5834C122542
:100E60000646236801226946284698479DF80000F7
:100E7000012240F008008DF80000636869462846AA
:100E800098474825236801226946284698479DF8D7
:100E90000000012220F0060040EA46008DF8000024
:100EA00063686946284698472368012269462846B0
:100EB00098479DF80000012240F001008DF80000E5
:100EC0006368694628469847F8BD38B5674D482499
:100ED00001222B686946204698479DF800000122B0
:100EE00020F001008DF800006B68694620469847A5
:100EF00038BD38B55D4D2A2401222B68694620464D
:100F000098479DF80000012220F0100040F00100F9
:100F10008DF800006B6869462046984738BD38B5A3
:100F2000524D2A2401222B686946204698479DF895
:100F30000000012220F001008DF800006B68694676
:100F40002046984738BDF8B5484C442506462368E6
:100F500001226946284698479DF80000012240F08A
:100F600082008DF8000063686946284698472D2561
:100F7000236801226946284698479DF8000001220F
:100F800020F0FC0040F08E008DF800006368694698
:100F90002846984714252368012269462846984721
:100FA0009DF80000012220F0070040F001008DF8BC
:100FB0000000636869462846984715252368012282
:100FC0006946284698479DF8000006F01F0120F06A
:100FD0001F0001438DF8001063680122694628460E
:100FE0009847F8BD2DE9F843204C1325174688464D
:100FF00081462368012269462846984701269DF8C4
:10100000000006FA08F120F01F0001F01F01014363
:101010008DF80010636832466946284698472725B0
:10102000236801226946284698479DF80000BE4083
:1010300020F03F0006F03F0101438DF80010636887
:1010400001226946284698472E25236801226946D1
:10105000284698479DF80000012240F00C008DF8CA
:101060000000636869462846984705E01C031000A5
:10107000380210003F0C00003E2023680122694620
:1010800098479DF8000000F0300189F80010BDE895
:10109000F883554B40F480701B681847524B40F45E
:1010A00080705B68184701B506209DF8001001228A
:1010B00001F01F018DF800104B494B6869469847B5
:1010C00008BDFEB5494D0446007828706078687008
:1010D000454EA078A870312733680122694638460A
:1010E0009847E07940069DF8000002D540F02000C6
:1010F00001E020F020008DF80000E179090602D51A
:1011000040F0800001E020F080008DF8000073685E
:10111000012269463846984721893220C1F30801E7
:10112000ADF80010E168CDF8021029788DF80610AE
:1011300069788DF80710A9788DF80810736809226E
:1011400069469847FEBD70B504460168274886B0D9
:10115000254D8160A168C160E1680161217C162094
:1011600001F001018DF80010617C8DF80110A17C67
:101170008DF8021000218DF80310A18A0F22C1F30F
:101180000C01ADF80410E18AC1F30B01ADF80610B3
:10119000218BC1F30B01ADF80810618BC1F30B017A
:1011A000ADF80A10A18BC1F30B01ADF80C10A17FB3
:1011B0008DF80E106B686946984731262B6801221E
:1011C00004A9304698479DF81000E17F20F01F00E9
:1011D00001F01F0101438DF810106B68012204A972
:1011E0003046984706B070BD1C031000380210004E
:1011F0004FF0E0214FF48030C1F88001C1F8800247
:101200007249A02081F80004704730B5704C012568
:101210002560E50603F03F0385F86B30002304E00A
:1012200051F8235040F823505B1C9342F8DB002018
:10123000206030BD30B595B00446302104F052FC3A
:101240006448006800906348001D00680190614890
:101250000830006802905F480C30006803905D48D9
:101260001030006804905B481430006805905948BD
:1012700018300068069057481C30006807905548A1
:101280002030006808905348243000680990514885
:10129000283000680A904F482C3000680B904D4869
:1012A000303000680C904B48343000680D9049484D
:1012B000383000680E9047483C3000680F90454831
:1012C0004030006810904348443000681190414815
:1012D0004830006812903F483F494C306FF002059B
:1012E00000681390009888424DD1A810A061206139
:1012F0002060A062E062E061206203A8029900F031
:101300006FF8019981423ED10B9845F2AA5180B203
:10131000884208D10498C0B2A061139A92B28A425E
:1013200000D0801DE0610C9880B2884217D10398EC
:10133000039A00F47F40D2B240EA0240039AC2F31B
:1013400007421043254A904203D30598C0F3012079
:1013500000E000202061059800F00F0020600D984B
:1013600080B2884201D10698A0620E9880B288426D
:1013700001D10798E0620F9880B2884201D10898A5
:10138000206215B030BDA56125612560A562E562CA
:10139000E5612562F5E710B50446142104F0A2FBCF
:1013A0000C487C38006820600A488038006860601B
:1013B000084878380068A060064874380068E06023
:1013C000044870380068206110BD000010E000E0A3
:1013D000441B0022B41E04005C000D6000010200EA
:1013E000F0B5074600200346184E10E057F823508A
:1013F00003224FEAC20C45FA0CF484EA2064E4B2FA
:10140000521E56F8244084EA0020F2D55B1C8B4221
:10141000ECDBF0BD70B5054600200C4C0246103CDC
:1014200009E0AB5C521C03F00F0604EB1313A65D3E
:101430001B78304418448A42F3DB70BD08B5009035
:10144000401E00900028FBDC08BD0000B85C0000D6
:101450004FF00051C88C4C4A00F0030012687AB17A
:1014600001280AD0022806D0032802D04FF41670B3
:101470000EE046200CE096200AE04FF4967007E05C
:1014800001280ED002280AD0032806D04FF4E170BC
:10149000401E21F8520F088070473220F8E76E2076
:1014A000F6E7DC20F4E748F61971480720F82A1F10
:1014B0000B2180F83E1000214183022180F8C010EA
:1014C0004FF008510120C1F8D4032F499839086022
:1014D0002E49086070474FF0005141F29840C8848F
:1014E000B6E74FF0005140F29A70C884B0E74FF071
:1014F0000050C08CA0F5A051983901D00020704751
:10150000012070474FF000518A8C60F304028A84F6
:1015100070471F48016841F00401016070471C4892
:10152000016821F00401016070474FF0005108810B
:101530007047174928310968016015491831096851
:10154000416013491C3109688160114920310968E3
:10155000C1600F492C31096801610D490C390968D6
:1015600041610B4914310968816170474FF00050A7
:10157000808870474FF00050807970474FF00051DD
:101580004C2081F820007047DC040022EC1B002274
:1015900010ED00E030B41DC8484981E81D0001216C
:1015A00030BC002004F026B82DE9F84F444801244F
:1015B000006810F86C5F417890F846004D4300F0E9
:1015C000030004FA00FA3D486421103004F08AFA5E
:1015D0003C4803F0B3FB3B483B490471097809B927
:1015E00002210171DFF8D480002408F1100B36E0ED
:1015F000DFF8D090032735490026C9F80010484687
:1016000003F0A0FB00226B460121104604F042F8D3
:101610000121002004F01DF898F8000060B102F0EC
:1016200058FD7F1E002F0AD0E9DC76B34FF0000092
:101630005946D8F804200FE04FF00106F5E74FF0C7
:10164000040003F074FBF0E751F8203032F9107019
:101650003B4441F82030401CA842F5DB641C544553
:10166000C6DB012E11D1164900205C46184A0B68D2
:1016700009E093F8B26054F8201006F003063141F7
:1016800022F81010401CA842F3DB12490120087018
:10169000BDE8F88F10B50446002004F05CF8022085
:1016A00004F059F8E00701D0FFF77EFF022004F0B4
:1016B0006DF8BDE81040002004F068B83403100055
:1016C000E40210004C021000090310004515000050
:1016D000664101209002100010B51C4C40F2FF1131
:1016E0002068FFF77DFE2168C1F8FC07FFF748F886
:1016F00000213F200EF1ACFAFFF742F82168BDE867
:1017000010403F234FF400721148FFF77EBD10B523
:1017100040F2FF310F48FFF763FE0E49C1F8FC0F9E
:10172000FFF72EF800213D200EF192FA00213E2015
:101730000EF18EFAFFF724F8BDE810403D234FF478
:10174000806204490448FFF760BD0000E402100015
:10175000F0EF03004C000120F0CF030030B41DC8AF
:101760004F4981E81D00012130BC002003F042BF39
:1017700010B5002003F0EFFFFFF7BBFB00F064F8AB
:101780000446FFF7CCFB012C04D13C224549A020A4
:10179000FFF77FFC002003F0F9FF012010BD10B51A
:1017A000FEF714FFBDE81040822002F0A5BC2DE931
:1017B000F047002003F0CFFF00253B4F4FF0360AE3
:1017C0006E1EA846E8B2FFF76EFC0020FFF745FB4F
:1017D0003C683868A042FCD03868A042FCD133494C
:1017E0006420FEF7FBFEFEF79EFF81463868A042AC
:1017F000FCD03868A042FCD1FEF795FF0446FFF705
:1018000064FBFEF7E3FEA9EB040080B2B0EB0A0034
:1018100001D4014600E04142B14204D2002800DA7E
:1018200040420646A8466D1C6DB2202DCADB1D49FC
:1018300008F0FF00743981F8B000FFF734FCBDE810
:10184000F047002003F0A2BFFEB50025684603F074
:1018500075FA174800900320114E8DF804000446D5
:10186000684603F06FFA002202AB0121104603F034
:1018700011FF0121002003F0ECFE307838B1641E26
:1018800002F027FC002C05D0EADC2846FEBD4FF014
:101890000105FAE74FF0020003F049FAF5E700000E
:1018A000A8031000C0000120981B00224F17000061
:1018B0000D17000030B41DC88E4981E81D000121BC
:1018C00030BC002003F096BE2DE9F84F8A4800682E
:1018D00010F86C4F40784443FEF75FFF8548642161
:1018E000103004F0FFF83221844804F0D9F8322196
:1018F000834804F0D5F8814842F21071323004F088
:10190000CFF8DFF8F8A10020AAF1320A47F6FF71FC
:10191000AAF1320BCA4304E02AF810102BF8102069
:10192000401CA042F8DB774803F008FA7549012013
:1019300000250871DFF8CC9103267349DFF8B481E4
:101940000027C9F80010484603F0FCF900226B4656
:101950000121104603F09EFE0121002003F079FED4
:1019600098F80000C0B102F0B4FB761E002E16D02D
:10197000E9DCBFB36148D8F8041005FB04F200F1BC
:101980003200DFF8708100EB42034FF00000564652
:101990005F4608F1100823E04FF00107E9E74FF038
:1019A000040003F0C4F9E4E731F8102023F8102014
:1019B00058F8202031F910C0624448F8202031F94D
:1019C000102037F910C0624501DD27F8102031F9E9
:1019D000102036F910C0624501DA26F81020401CAC
:1019E000A042E1DB6D1CC82DA4DBDFF808810020DC
:1019F000C821424D52465B4608F110080EE033F90B
:101A0000106032F91070F61B761025F8106058F847
:101A1000206096FBF1F648F82060401CA042EEDB07
:101A2000364F0020364E3237894615E0002258F8EE
:101A30002030114601FB040C37F91CC0BCEB030C31
:101A400001D5CCF1000C491C6244C829F2DB92FBA1
:101A5000F9F126F81010401CA042E7DB002707E050
:101A600036F9172035F91710F8B202F031FD7F1C56
:101A7000A742F5DBBDE8F84FFEF782BE2DE9F8433B
:101A800000248DF80040FEF788FE002003F063FE7E
:101A9000194D286890F86B00FFF755FA2F6800255C
:101AA000A1464FF00108A1370024785D08FA04F63A
:101AB0008DF8009006400DD0224629466846FFF773
:101AC00091FA9DF80000202804D1324629460520CD
:101AD00002F0FBFB641CE4B2062CE6D36D1CEDB2F5
:101AE000052DE1D3002003F051FEFEF749FEBDE8CD
:101AF000F8830000B8031000E4021000B0100120C9
:101B0000F2370120540210006518000010B5044699
:101B10000221002003F06EFD0F48046010BD08B5DF
:101B20000E48FEF74EFE00226B460221104603F0DF
:101B3000B1FD0221002003F08CFD09485522016807
:101B400005480A7100684871020A8A71020CCA715C
:101B5000FEF7E7FC08BD00005C021000BD1A0000A3
:101B6000E802100008B50024DFF85881564F4FF402
:101B70000049264600226B464146104603F08AFD86
:101B80000098800319D5FEF741FC504804680660B0
:101B9000FEF73AFCE00701D0FFF709FEA00701D5E8
:101BA000FFF7E6FD00231A460121022002F077FC30
:101BB0004FF40031002003F04CFD0098000411D5D3
:101BC00000256D1CEDB2FFF7D3FD01286ED0032D6B
:101BD000F7D900224946082002F077FB4946002049
:101BE00003F037FD0098000510D5394804680660F9
:101BF0002046FFF74FFD4FF40061002003F029FD60
:101C00000023E1B21A46062002F049FC0098C00405
:101C10000CD5FFF784FF002301221946022002F0B1
:101C20003EFC4FF48051002003F013FD0098800427
:101C300006D5FFF751FD4FF40051002003F009FDD8
:101C40000098400406D5FFF762FD4FF48041002064
:101C500003F0FFFC0098400311D5386890F8A0000D
:101C6000C0070CD0FFF70AFF4FF48021002003F0DB
:101C7000F0FC00231A4619460C2002F010FC0098D4
:101C800000037FF577AF386890F8A0008007F8D59B
:101C9000FFF71AFE4FF40021002003F0DAFC0023C6
:101CA0001A4619460E2002F0FAFB63E70120FFF7FF
:101CB000F1FCE1B20023C4F30722082002F0EFFB9D
:101CC0008CE7000003F80F00E4021000040310008A
:101CD0000003100010B58143C80711D064480168A3
:101CE00041F0010101604FF40061002003F082FC2B
:101CF00001220023BDE810401146052002F0CFBBB1
:101D000010BDFEF7F2BC10B5FEF7EFFC0121BDE8F7
:101D10001040084603F06EBC5649012805D0022841
:101D200005D0032805D1042002E0022000E00320B2
:101D30000870704738B5002003F00DFD4E4800686C
:101D400010B1FFF7E9FF01E000F0CCF949484B4939
:101D50000078022813D003280ED0042812D00124C2
:101D60000025FEF7D6FE00B101256946032003F0E9
:101D700080FC009858B909E00868847AF0E70868A0
:101D8000447AEDE70868B0F80B40E9E715B1142C88
:101D900000D2142420463A49FEF7AFFC0324394D03
:101DA00000F022FA012807D1287858B1641E02F009
:101DB00090F9002C0DD0F3DCBDE838404FF0000066
:101DC00003F0E4BC304801683048006800F01CF9BA
:101DD000F2E7032002F0ABFFEEE770B52C48046891
:101DE0002C490D680C6095EA040F27D0214E2DB1C7
:101DF000A4B121462846BDE870406BE70220307050
:101E00001E4800680079000701D404203070214684
:101E10002846FFF75FFFBDE870408BE7FEF765FCE3
:101E20000121084603F015FC0120307021462846A8
:101E3000FFF750FFBDE8704000F0F7B870BD10B577
:101E4000FEF753FC0121084603F003FC0949042076
:101E5000087000F0B1F8BDE810406BE710B5FEF770
:101E600044FC0121084603F0F4FBBDE8104061E7A3
:101E70000003100070021000F8021000E4021000CD
:101E8000B71C00002C0410007C0210007802100027
:101E9000F0021000740210002DE9FC5F0E460028CD
:101EA0001BD055490978042917D1002A15D1DFF82C
:101EB0004C91DFF84C81534DD9F800109246097AC5
:101EC00049070ED5A978491CC9B2A970032906D8BB
:101ED000018808EB460020F8021CBDE8FC9F85F84D
:101EE00002A0032003F037FC454801906C78B5F957
:101EF00004B02878274640B941480F235A46009439
:101F0000801D019902F038FD002734B93C4A5B4638
:101F1000921D901D019902F020FD39496F700C311E
:101F2000B5F90420B5F90630002007E031F910407A
:101F30009C4201DD012404E0401CC0B29042F5DB6C
:101F40000024032003F022FCD9F8000090F8E307F6
:101F5000DA2823D1D8F80010C8F81210B8F8041005
:101F6000A8F81610D8F80610C8F81810B8F80A1013
:101F7000A8F81C10D8F80C10C8F81E10B8F81010EB
:101F8000A8F822101E48C8F824A0C8F828A01230CB
:101F9000A8F82CA04682A9788182C4822C70002CDB
:101FA0009BD0FFF7AEFEBDE8FC5F0121084603F0C1
:101FB00021BB144800787047124A012050700F4826
:101FC0000068017A4B0790F8711002D590F86C30D8
:101FD00001E090F8703059439180B0F84B00D08008
:101FE0000021074811709170C1600182C0F806108D
:101FF000418100F0A9BADFE770021000E40210008E
:10200000243801206002100070B5054630480C46A7
:10201000224690F90D102F484068FFF73DFF2146FA
:102020002846BDE8704000F014B810B5032003F056
:1020300092FB4821284803F055FD274901200870EC
:10204000032003F0A3FB0121BDE81040022003F0B0
:10205000D1BA2DE9F041DFF884800746002698F8D0
:1020600000000D4604282CD047EA0504032003F0A5
:1020700072FB194A174B978115619868506098F860
:10208000000004281FD0FF2111751070E0070DD04B
:102090001348016811F86C0F49784843906042007A
:1020A0000D485968163003F07CFC0126032003F02C
:1020B0006DFB002E09D0BDE8F0410121022003F0A4
:1020C00099BA0C46D2E7197BDEE7BDE8F081000043
:1020D000500610002C04100094061000700210002E
:1020E000E40210002DE9F0417A4C0026DFF8E88187
:1020F00020780227794D04280ED000F005FF012832
:1021000019D07748237802680320022B517B10D125
:1021100098F8003093B113E0FFF74BFF012803D08C
:1021200098F80000012804D16E49277001202E6024
:102130000870BDE8F08127702E60FAE7917B0420DB
:10214000127AD30701D19207F3D52A68521C2A606C
:102150008A42EEDD2E602070EBE730B41DC8624984
:1021600081E81D00082130BC012003F043BA2DE9AD
:10217000F0415B4800240068C17BC90732D05B494D
:10218000564E27460978C90727D0DFF84881012431
:1021900098F8001002290BD004290BD0857C00F0A0
:1021A000B3FE012808D05248007801280BD00EE079
:1021B000457CF4E7C57CF2E798F80000042806D0D7
:1021C0000024776006E098F80000022807D07068C5
:1021D000401C70607068A84203DD776002E07760A1
:1021E000F8E700242046A4E72DE9FE4339483F4D97
:1021F000012600783F4FDFF80081032816D004281D
:10220000684610D0002402F099FDFFF7B0FF29784E
:10221000C90700D0012440EA0401C90716D02E499D
:10222000097801B310E000F02EF812E068460024AF
:1022300002F084FDFFF79BFF2978C90700D0012435
:1022400040EA0401C90701D08DF804603860C8F87D
:1022500000402A480090684602F074FD012806D02C
:102260000020BDE8FE8302218DF80410EEE702ABEA
:1022700000220821012003F00DFA0821012003F0BB
:10228000E8F90120EDE770B50446002502F056FD9F
:10229000FFF76DFF1249C3074FF0020205D009682E
:1022A000C97B89070FD504210BE0104B1B78DB0796
:1022B00000D00225AB0707D50968097A490702D57E
:1022C0000521217100E022710A4908600A48056071
:1022D00070BD0000700210000903100068021000B9
:1022E000E4021000900210002C0410007402100090
:1022F000EC0210007C021000780210000B2100009C
:102300001C4808B500210122416002708160C16053
:10231000491E104603F09DF9FFF76DFE6B46002243
:102320001721012003F0B6F90098800705D5FFF7C3
:1023300054FD0221012003F08CF90098C00705D05C
:102340000121084603F085F9FFF7F4FC00984007E7
:1023500005D50421012003F07CF9FFF770FD0098FA
:10236000C006DBD51021012003F073F9FFF776FDDD
:10237000D4E700007002100032216E4803F090BBD9
:102380002DE9FC5F88466C4905466FF0130208682A
:102390004FF0010AC446037CB0F9167003F00F0435
:1023A000B0F91A30C4F11006B8F1280F15DB8B46CE
:1023B0004FF00009C18ACDE90019838A28223C2107
:1023C000604602F0B8F907B2DBF800002822418B22
:1023D000CDE90019038B3C2118E008F1140CBCF185
:1023E000140F17D84FF00109C18ACDE90019838A6B
:1023F00093460021404602F09EF907B24E48002164
:102400000068428BCDE90029038B5A46404602F012
:1024100092F903B24948DFF81CC1006881460AE01E
:102420003CF9101035F9102001EB0708904515DB39
:10243000C91A914212DC401EF2D2BAF1000F0DD03F
:10244000494609E03CF9112035F91100624300FBCF
:10245000062000112CF81100491EF3D2BDE8FC9FA4
:1024600070B514460D46C00716D000F04DFD00288B
:1024700012D131480068C07B800703D5304800780E
:10248000042804D021462846BDE8704078E7284655
:10249000BDE8704000F001B870BD2DE9F04F26494D
:1024A000284C4FF0010E0A68DFF888B094F900401C
:1024B000117CB2F916A001F00F0692F86D10C6F16A
:1024C0001008B2F91A900B4614E093FBF1F7C3EB36
:1024D000440501FB1737EDB2FFB23BF9155030F957
:1024E000177005EB0A0CBC4522DBA5EB0905BD42C4
:1024F0001EDC5B1E012BE8DABEF1000F18D0DC46B3
:1025000014E092F86D50C1EB440391FBF5F705FB25
:102510001715EDB2DBB230F915703CF91350754365
:1025200007FB08552D112CF81350491E0129E8DA34
:10253000BDE8F08F66410120E4021000AC021000FB
:10254000A8021000A902100070B5FE4C00256421FD
:10255000C4F80B50FC4803F0A3FAFB486421643034
:1025600003F09EFA6570A5704FF4F071F74803F020
:10257000B9FAF64E00216FF0004301EB810006EB43
:102580000012002042F82030401C1428FADB491CBD
:102590000629F2DBE570EB4AA4F805500020032180
:1025A000E57108321154401C0328FBDBE64840F279
:1025B0001451C83003F074FA257170BDF0B4E44CC6
:1025C00000231A462478022C02D0F0BC184670472B
:1025D000E04B1C68E04B1E6874B900230AE030F938
:1025E000134096F8C950AC4201DCEC4201D50122FF
:1025F00002E05B1C8B42F2D396F8B710F0BCD148D6
:102600000D3000F0F3BB2DE9F04F87B091464FF04D
:10261000000A3C22D04BCDE903A21A6892F8B040E0
:10262000A40600D51098C84B02F5AB7592F8B860B7
:10263000AC1DC8338E4211DC92F8B9608E420DDBBE
:10264000B2F87E11A51D4942009101910291B3F8A3
:10265000E4140C34491CA3F8E41420E092F8C86098
:1026600076428E4210DB78210491B2F87C1102F59B
:10267000B7754942009101910291B3F8E614AC1D7F
:10268000491CA3F8E6140AE0B2F87A114942009115
:1026900001910291B3F8E214491CA3F8E214AA498B
:1026A0002A88C831DFF8A4E2A1F8E8242288A1F83A
:1026B000EA246A88A1F8EC246288A1F8EE24AA88AA
:1026C000A1F8F024A288A1F8F2249E4A0021D37830
:1026D00046E0CA070DD001EBD172521002EB820224
:1026E00003EB82060EEB860230F9117016683E4449
:1026F0000CE002290CD001EBD172521002EB8202E5
:1027000030F9116003EB82070EEB8702166003E0DD
:1027100003F114064EF826A001EBD172DFF824C2B3
:1027200056100CF1080C06EB86080CEB620B03EB61
:1027300088079BF800205EF827707646032A0ED1A2
:102740004FEA72020A40012A09D1002202EB880CEA
:10275000521C46F82C70142AF8DB8BF800A0491C98
:102760004945B6D300203FE000EB80030EEB031693
:10277000744B0596002193F803B00A464FF01408F5
:10278000ABEB020707F1140393FBF8FC08FB1C33C7
:10279000521C56F823C007F11E0393FBF8F708FB01
:1027A00017330A2A56F82330ACEB03031944E7DB4E
:1027B000644B06F1F002083342F82B101A5C12B198
:1027C000012A06D00FE035F810208A420BDA0121E9
:1027D00008E034F81020CA4205D55A4A521D022199
:1027E00002F800A01954401CB0EB590FBCD30020D4
:1027F00081E0544B00EB800447F6FF710EEB0416AA
:10280000CA430024DD7814272B1B143393FBF7FCF9
:1028100007FB1C3356F823308B4200DA19B293427F
:1028200000DD1AB2641C0F2CEEDB464C0834235C2E
:10283000012B02D0022B15D05CE0531A00D55B426D
:10284000454D2D6895F8BE50AB4253DC5DF8203005
:102850008B424FDA002B00DA5B4293424ADD04F8E8
:1028600000A047E0DFF8DCB0049B0BF1050B1BF880
:1028700000C09C454AD200242B1B143393FBF7F86D
:1028800007FB183356F823308B4200DA19B2934213
:1028900000DD1AB2641C0F2CEEDB531A00D55B422C
:1028A0002D4C246894F8BE40A3421FDC5DF8203014
:1028B0008B4206DA002B01DB1C4600E05C428C42B6
:1028C00006DC93420EDA002B00DA5B42934209DD0C
:1028D0001C4A03210832115451460BF800A003AAE8
:1028E000115407E003A901220A5403E00CF1010C82
:1028F0000BF800C0401CB0EB590FFFF47AAF174A39
:10290000002003AD295C012906D00EE00D4A514696
:102910000BF800A00832E3E7012863D0109902EB1E
:10292000800301EB800109681960401CC0B20328D4
:10293000E8D3054B03490020C8331924F34609792D
:10294000004A0DE0800210004E3801203C041000C7
:10295000090310009C021000E402100066410120EF
:10296000D5780022192901D340F24512B1FBF4FCBD
:1029700000EBC00606EB001602EB860200EB8007B8
:1029800004FB1C1C0BEB071707F1F006944437F807
:10299000257023F81C7056F825700A2697FBF6F66A
:1029A000B1FBF4F704FB1717174403EB47070DF1CE
:1029B0000C0E7E861EF80060012E18D0F94E375C92
:1029C000B1FBF4F604FB1616164447B303EB460CB2
:1029D000461C40F2712806FB08F607EB0616ACF819
:1029E000646020E01099F04BC988D9809DE7B1FB65
:1029F000F4F604FB1616164403EB4607461C40F299
:102A0000574C06FB0CF6A7F86460B1FBF4F704FB27
:102A100017173A4403EB4202A2F896600FE003EB6B
:102A20004607A7F864A0B1FBF4F604FB161632447F
:102A300003EB4206DB4AD21E125CA6F89620401C2D
:102A400003288EDB002047F6FF7503EB4002401C95
:102A5000A2F858521928F8DBD24F3220083F491CFF
:102A6000B1FBF0F200FB12123A71002040F2451661
:102A70000021192A00D33146B2FBF4F700EBC00C59
:102A800004FB17270CEB001C67443944401C23F857
:102A900011500C28ECDB0023DFF8088318466FF098
:102AA0000042564601254FF0030CA8F1030715E03C
:102AB0001EF8001000EB80040BEB041401290CD16C
:102AC000002144F82120491C1429FADB05FA00F101
:102AD00008F800C019433E54CBB2401CB0EB590F6C
:102AE000E6D323B114220121052001F0D8FCAD4A20
:102AF0001421083AD078401CB0FBF1F301FB13001D
:102B0000D07007B00020BDE8F08F2DE9F04F8FB0F6
:102B10008346A64A00200E9012688846BBF904102E
:102B200092F8B520914250DDBBF9062091424CDD70
:102B300000244FEA58000D90DFF874924FF0FF3AEE
:102B40002746264625463421684602F0CBFF4246FA
:102B50005946684601F0D0FD944900206B460A684A
:102B60001BE033F91010B0EB580F08D292F8B6C042
:102B7000614511DC761C2144F6B20CB20CE092F8EF
:102B8000B5C0614508DD6D1C0F44EDB23FB249454B
:102B900002DD89460FFA80FA401C4045E1D3BAF1C4
:102BA000030F0BD10D98864208D1854206D1002C27
:102BB00000DA6442BC4201DA01200E90794892F8B2
:102BC000B710001D0E9A00F011F90FB09BE7F0B49A
:102BD000764A00252C462E46136813E0022911D0B0
:102BE00030F91120B3F8CE70BA4202DD15442DB28F
:102BF00002E001DA144424B2DF8AC7F10007BA42C6
:102C000000DA0126491EE9D2002C00DA6442654848
:102C1000C01CAC4204DD1EB193F8CB10012202E0CF
:102C200093F8CB100022F0BCC01C00F0DFB82DE9F7
:102C3000FF4F81B007469B469246002402200E9E1D
:102C400002F089FDDFF86491564DD9F80000A5F136
:102C5000080590F8B000C0060ED55648007858B167
:102C600053463246594618460097FFF7CCFC0446B7
:102C7000012801D1142028704A480027017819B989
:102C8000417809B9807838B1C5F80B70022002F09C
:102C90007DFD002005B036E744BBD9F8002092F84E
:102CA000B000C00725D04FF0000CD046614660460A
:102CB00008E038F9103092F8B340A34201DD491C16
:102CC000C9B2401CB042F4D3B14201D14FF0010C63
:102CD000344892F8B4106246C01C00F087F80446ED
:102CE000012804D02F48C01C077014B121E0102027
:102CF00023E0D9F80000C84690F8B00040060AD595
:102D0000F1B25046FFF763FF0446012801D014B129
:102D10000FE0152011E0D8F8000090F8B00080070F
:102D200013D531460298FFF7F0FE0446012803D080
:102D30005CB1012C02D003E011202870C5F80B70A3
:102D4000022002F023FD2046A4E7D8F8000090F806
:102D5000B0000007F4D572B259460298FFF72EFC76
:102D600004460128ECD11320E7E770B506460F4D65
:102D70000C7800200870286890F8B100C0071FD0B8
:102D8000022002F0E8FC0C48314600684200064888
:102D900002F007FE094801210170022002F0F6FC52
:102DA00018E000008802100066410120E4021000D3
:102DB0000080FFFF09031000AC0210009002100019
:102DC0001248016841F0010101604FF400610020E8
:102DD00002F010FC28682246012190F8B100BDE8FD
:102DE000704000F00103052001F059BB10B500232D
:102DF0001C4642B10278521CD2B202708A4203D9F8
:102E00000470012300E00470184610BD0003100098
:102E100010B5FF4C012019212070FE4802F062FE1F
:102E2000FC4832211A3002F03BFEFA4832214C3085
:102E300002F036FEF7490020083948602061E06062
:102E400060704FF4C8706061BDE810404FF4967137
:102E5000F14802F025BEF0B5F048F14C01220168BE
:102E60000020206060602081C4F80A00C4F80E00D1
:102E70006082EC4801F13F0301F147060778EA4818
:102E80000078384303D1E948007800B10222DFF826
:102E900090C300200CF10A0C0EE033F8105055439B
:102EA00024F8105033F8105016F800E0A5EB0E058A
:102EB00055432CF81050401C91F86C508542ECDCC6
:102EC000002F0AD0DA480078002806D1D14831F81E
:102ED000632F0838028089784180F0BDCF480068B0
:102EE00090F8801069B1490010F88C2F521C40787E
:102EF0004A43C2EB022100F01F000141C448C180D7
:102F000070470121F0E77047C1480069002800D0F0
:102F1000012070472DE9F04FBD4D4FF0010A0AFA2C
:102F200001F6ED68DFF8ECB22E40C04DABF1080BB6
:102F3000DDE909EC2F78BB4D4FF00009BBF80080AC
:102F40002D784C460BD025B1BBF80240A8EB040409
:102F5000A4B2BCF1010F0CD05DB157B10DE00DB1C1
:102F600007B14446BCF1000F01D105B12FB9AC4CFB
:102F700001E0AB4C0A3434F81140A84D2D6895F8A7
:102F80003A50ED0738D0BEF1010F0BD0012930D0F7
:102F900030F9135030F912108D4200DD2946A1425C
:102FA00033DC38E030F91250002D06DD30F9131013
:102FB000002902DD294409B204E030F91310A942C6
:102FC00000DC294656EA0C070CD0002EE7D0BCF1F5
:102FD000000FE4D1A542E2DA30F91300A042DEDAB4
:102FE0000021DCE7A542DADC30F91300A042D6DC90
:102FF000F6E730F91310D2E730F9121076B1A1429A
:1030000009DA30F91300A04205DA0AFA02F00AFAE6
:1030100003F141EA00094846BDE8F08FA142F4DC23
:1030200030F91300A042F0DCF5E72DE9F041154638
:103030000024621E794E8EB08046012941D1342190
:10304000684602F04FFD7B4F414668463A6801F002
:1030500053FB397840F6FF7268462B6800F0F4FBAA
:103060006B49024628680B7B20EA0303DB0708D084
:103070003368B3F84F30934203DD20F001000124A0
:10308000286083070BD50B7B9B0708D43368B3F804
:103090005530934203DA20F00200A41C2860430755
:1030A0000FD5097B49070CD43168B1F857309342EA
:1030B00003DCB1F85910914203DA20F00400241D1A
:1030C0002860306890F8E307DB2808D1002C06D090
:1030D0000EB02146BDE8F041FD2001F0DFB80EB092
:1030E000BDE8F081014600208A0700D0012011F0E0
:1030F0000C0F01D040F0020011F0300F01D040F071
:103100000400704730B4117889073DD5B0F9043018
:10311000B0F906108B4237DD002B00DA0023B0F93E
:103120000040002C00DA0024B0F90850002D00DA2D
:1031300000252C44C4EB43031BB2002900DA002114
:10314000B0F90240002C00DA0024B0F90A0000288F
:1031500000DA00202044314CC0EB410000B221686D
:10316000B1F84D10994201DC81420DDD0021116062
:10317000216891F8E317DB2906D140EA03420121D7
:1031800030BCFC2001F08AB830BC7047FCB50C465E
:103190000125CDE900540746052304220221FFF74B
:1031A000B9FECDE9005406460022012311463846F7
:1031B000FFF7B0FE40EA06050020CDE90004032336
:1031C000022201213846FFF7A5FE2843C0B2FCBD0C
:1031D0002DE9F0410C46014632220F4802F0E1FB96
:1031E0000D4832221449323002F0DBFB09490A480B
:1031F00032221A31643002F0D4FB064906483222EA
:103200004C31963002F0CDFB00204FF0010E15E05E
:1032100090021000343E012000EC0120E402100076
:103220001C06100018410120EC02100009031000D8
:1032300008031000AC02100066410120FF4AFF2382
:1032400007465668FE4AFC49156814E00EFA00F27B
:10325000224201EB400C02D0ACF8C83001E0ACF8DF
:10326000C870324201EB400202D0A2F8FA3001E00D
:10327000A2F8FA70401CA842E8D331E72DE9FC47D8
:10328000F04D8146ED488A4600262C782E7032217A
:10329000B83002F005FC14B1B9F806002881EA4FF5
:1032A000E74D386890F82A10C9070BD0009490F8C1
:1032B0002B00494600F00F03288802B2DF48223075
:1032C00001F05AFB022002F046FA2888DB4900B2DE
:1032D000223100905346DD4A01F1960001F088FA50
:1032E000022002F053FAD5493222B831A1F132005E
:1032F00002F057FB3868DFF85883C07B000715D50C
:10330000D4480078012811D198F8000070B9D2484B
:10331000007858B12888C94900B20090CF48B83128
:1033200002680846938E243201F047F92868C349A1
:103330004200B831A1F1640002F033FBC84998F8AB
:1033400000000978084330D1386890F82A00400717
:1033500007D5BA492A788631012301F1320000F0FD
:10336000A0FA386890F82A1089070BD590F86D10EC
:103370000091B24990F86C3090F82C20B831084692
:1033800000F00FFAAD493222B831A1F1320002F05B
:1033900008FB2868A94ACDE900045432534602F1DB
:1033A00032014846FFF743FC06463046BDE8FC873D
:1033B0002DE9F0410025A24B06462C46681E2A4600
:1033C000AE46DFF880C21F680CE036F912308B423F
:1033D00002DA0B44002B04DC012536F9124050B20E
:1033E00003E0521CBA42F0D3A5B19CF80110491C6D
:1033F000C9B28CF8011032290ED99A4A8CF801E032
:1034000001211160C3B2E2B2C4F30721ED2001F043
:1034100046F801E08CF801E0284661E68A4A10B5DA
:10342000126804460020128C891A0BB2844909687C
:1034300006E034F911209A4201DCDA4200D501207D
:10344000491EF6D210BD70B57F4D02460024286893
:10345000C07B40071CD51046FFF7E0FF012817D1BD
:10346000FCF7D4FF804C206840F002002060FCF79D
:10347000CBFF4FF40041002002F0BCF8286822780E
:103480000121C07BC0F38003072001F008F801246C
:10349000204670BD30B56B496B4B0022CD681B6870
:1034A000002D14464FEAC07505D07DB185070DD5B6
:1034B0008D782DB10AE04DB1850707D58C7005E0F8
:1034C00001258D700C7193F89750CD7010B18C78E8
:1034D00034B901E08C700C71024693F89700C87003
:1034E000104630BD10B5574CA078002805D0E078C4
:1034F00020B1401EE070207910B910BD012020716C
:103500004E480321007901F0F5FA0020A0702071E7
:1035100010BDF0B5554C4B4F0E4620780025A8B194
:10352000B6F90600B7F90810081A00D54042464916
:1035300000B20968B1F86010814207DA00204C49F6
:103540002070022001250870FFF785FC387821786B
:10355000084301D1F08838812846F0BD2DE9F047B5
:1035600004463648DFF8DC90344F4568D9F810003F
:10357000002384EA000834484FF0010A083706683F
:1035800020E00AFA03F010EA080F10D0204220D001
:1035900023B1012B02D096F83DC006E05FEA817CA2
:1035A00005D05FEAC47C96F83BC007F803C017F962
:1035B00003C0BCF1000F0FD0ACF1010C07F803C041
:1035C0005B1C1BB29342DCDB2846C9F81040BDE807
:1035D000F08796F83EC0E8E7204201D00543EFE7C8
:1035E0008543EDE72DE9F34F81B0164D002400949B
:1035F0008346B5F90610FFF7DBFE012845D0A84643
:10360000B5F906105846FFF71EFF01284BD0584663
:103610000299FFF733FE0446012850D002F020FB48
:1036200001284CD00548134ADFF81C908630106002
:10363000D9F80010C97B1FE000EC01202C3E0120CE
:10364000AC02100090021000E4021000664101205C
:10365000EC0210001841012009031000E8021000DC
:10366000ED021000F8021000040310000A0310001D
:1036700080021000C0021000A94FAA4E090724D5ED
:10368000A949097801291CD01FE0A8480068012831
:1036900008D168694FF00051401E686111F8360F7B
:1036A00003D008700020BDE8FE8F40F002000870D3
:1036B000887820F0020088709D480460FDE720466D
:1036C000F1E7397809B99B49116030600021106831
:1036D000FFF75CFD050006D0387820B9012130687D
:1036E000FFF754FD05402846FFF7FCFC009004213D
:1036F0006846FDF78FFE904900F0FF0A3878097898
:10370000084317D1D9F800004D4690F83A00400719
:1037100004D56A4651463068FFF787FC286890F860
:103720003A00800706D5009820B16A4651463068B5
:10373000FFF7E8FC03224646D8F80C100098FFF784
:103740000DFF07465946FFF7E4FE7A4D543DA8B1F8
:1037500000246C602046029900F0D1FE28792146B1
:1037600001F0C8F9012475480078042803D05846B0
:103770000099FFF72DFD6868F060A0E76868874250
:103780000CD0F8B26F60FFF785FE074628790299E2
:1037900000F0B5FE2879394601F0ACF9FFF7A2FE3A
:1037A000E1E72DE9FF4F9146864600250D9F46E053
:1037B00005FB07F00199012247F6FF7C01EB40066B
:1037C0006FEA0C040EEB400B13460021C9F1000A0E
:1037D00016E036F9110048450FDA50450DDD8445F5
:1037E00000DD8446844200DA0446002802DA4FF005
:1037F000000202E001DD4FF0000301F1010189B296
:10380000B942E6D352EA030009D012B1012A04D02A
:1038100004E0012B02D1204601E023B10020410049
:103820000BD0002107E06046F9E736F81120121AA4
:103830002BF81120491CB942F7DB6D1CADB203987F
:103840008542B5D3BDE8FF8F2DE9F0410024491E24
:1038500017468646CAB2A44626462546D80701D052
:1038600002220DE098070BD50124032208E03EF95F
:103870001400604502DD00FB04660544641CE4B2EC
:103880009442F4D985FB012386FB070102F065F819
:10389000002800DA0020791E884200DD084600B2C8
:1038A0001EE42DE9F04F00259B469AB0531EDFB26F
:1038B0002C462B460DF1340AE94611E031F913602C
:1038C00035445E1CB44695FBF6F629F81360FE1AE3
:1038D0005B1C31F91680444494FBFCFC2AF816C0AA
:1038E0009342EBDBBBF1010F01D1921ED2B24C46E9
:1038F00055460FE034F9123035F91260334403EBCA
:10390000D3735B101BB2002B04DD31F81260F31A85
:1039100020F81230521EEDD21AB0BDE8F08F000030
:10392000EC021000BC02100018410120F802100047
:103930005C090022803E0120ED02100070021000A0
:10394000384808B50021C1608160416001210170E3
:10395000354914200870FFF75BFAFEF70DFDFEF7FE
:10396000F3FDFFF7BBFA6B4600220121022001F0B4
:1039700091FE0098C007F6D00121022001F069FEF7
:1039800000F001F8EFE770B50025032001F0E3FE39
:1039900000F024F8234C244E207BC00705D096F974
:1039A00000102069FFF71EFE0546A06858B10220EE
:1039B00001F0D1FE96F900202169A068FEF750FDC4
:1039C000022001F0E3FE012D03D118492069FFF721
:1039D000CCF9BDE87040032001F0D8BE70B5114CA1
:1039E000134DE068B5F90C1080EA0102D20708D047
:1039F000C90702D0FFF70CFA03E0C00701D0FFF7B8
:103A000082FAB5F90C00E0602869A060A8686060DF
:103A100007481630206128782070287D607005489E
:103A2000606170BDA8021000FC021000800210004E
:103A300094061000803E0120094C00202060401CAC
:103A40002060FCF7AAFE00F04BFEFCF779FD08B9F8
:103A5000FDF75FFDFCF7BEFB01F0B6FB2068EEE76B
:103A6000C4021000E04900200860E0490860E04915
:103A700008607047D0214DF6C062BA2000F025BC26
:103A800070B54FF40063984202D2DA4C246807E024
:103A9000A0F5805080B24FF4805398420CD2D64C9F
:103AA00085189D4200DD1A1A002303E0CD5C1E1824
:103AB0005B1CA5559342F9DB70BDB0F5805F04D265
:103AC0000A460146CB48006808E0B0F5FE5F07D320
:103AD000A0F5FE5080B20A460146C74800F012BC6D
:103AE000704700F0A4BF10B54FF40051002000F063
:103AF0006EF90023BDE810401A461946032000F075
:103B0000CEBC10B54FF48041002000F060F90023D6
:103B1000BDE810401A461946042000F0C0BCB24966
:103B20000A6882430A600221012000F050B9AE49C0
:103B30000A6802430A600221012000F048B9FCF73C
:103B4000C8BFFCF7A1BF10B5C00711D0AB48002318
:103B50000222016841F0010101600121052000F00D
:103B60009EFCBDE810404FF40061002000F02FB92A
:103B700010BD10B50324FCF749FCA1480460FCF714
:103B800043FC002301211A46084600F088FCBDE8EA
:103B900010404FF40031002000F019B910B5002397
:103BA00001221946104600F07AFCBDE810404FF49F
:103BB0008051002000F00BB90421012000F007B96A
:103BC0008C4A904B0128126892F8E32709D002280A
:103BD0000CD0882A09D1197800231A46172000F042
:103BE0005EBC882AF7D0087818707047882AFCD104
:103BF00048781870EFE77E4A00230128136005D14A
:103C0000087810211060012000F0E1B870474FF4EF
:103C10008021002000F0DBB84FF40021002000F0EC
:103C2000D6B874480021006890F86800C00711D029
:103C300075480068827A12B1FF2A03D00AE0C27A7E
:103C40001AB107E0C27AFF2A04D196218172A52118
:103C5000C172012100231A46102000F020BC6A48DE
:103C600000210B4600680A468172C172202000F0D4
:103C700016BC10B50978654C002031B101212170C6
:103C800063490870FFF7E7F800E020700120FFF7B4
:103C90005AFF00232178BDE810401A469A2000F010
:103CA000FEBB10B5594C2278D2B9594A1278BAB134
:103CB000584A042809D000201070002321781A46A1
:103CC0009F20BDE8104000F0EABB534B08881880E5
:103CD00048885249088001201070FFF7BCF8ECE7D3
:103CE000494A00EBD070136820F0010203F1340060
:103CF00001F057FE00231A4621789C20E1E7434A51
:103D00001278002A0BD0012809DC3F4809780023EB
:103D100000681A4680F83A109D2000F0C0BB70473A
:103D200070B53A4C2278A2B1374D00EBD07626F030
:103D300001022B6803F1240001F033FE29687008AA
:103D4000002348842178BDE870401A469B2000F08B
:103D5000A6BB2F480078002811D1264B304A314CA1
:103D60001B6808E031F8105022F8105031F810505C
:103D700024F81050401C93F86C508542F2DC70BD62
:103D800070B5214A4D78431E14680A781D44543496
:103D9000202D02DBDBB2FF2108E0A318421E1846EB
:103DA000491C01F0FEFD00231A460121BDE87040C8
:103DB000992000F074BB30B41B4C00B1087820701F
:103DC0000023C1B230BC1A46A32000F068BB38B54E
:103DD0000C46054601F00EFC6946284601F049FCF8
:103DE000009A2242F8D138BDF0021000F40210000F
:103DF000F8021000E40210004C0001200003100043
:103E000004031000FC021000E8021000EC02100095
:103E100018410120080310002C3E01202E3E0120F5
:103E20001C06100026061000ED02100010B520211F
:103E3000664801F035FE6548FCF752FE6349401EB6
:103E400011F8012BA2F190031F2B01D8604A05E065
:103E5000A2F1C0030F2B06D85D4A803252F823200E
:103E6000BDE810401047B82A21D00DDCB02A13D08D
:103E7000B22A27D1032825D108888A78BDE81040C6
:103E800040BA1146FFF719BEFB2A17D0FC2A19D1F8
:103E9000BDE81040FFF735BE022813DD31F8022BD4
:103EA000BDE8104053BA821E1846FFF7E9BD02284C
:103EB00008D10888BDE81040FFF713BEBDE81040E8
:103EC000FFF711BE10BD0120FFF731BE0120FFF743
:103ED00026BE10B5FEF738FBBDE810400120FFF705
:103EE00032BE00F057BA3B4810B5017809B1022143
:103EF000017039483949006891F9003090F824215F
:103F00009A420CDD90F81C0191F90010884206DA03
:103F1000FEF71AFBBDE810400120FFF714BE10BDEC
:103F20002C480178002903D003210170FEF793BFCC
:103F3000704770B52A4D284C002028702068007802
:103F4000A52802D0012000F0C9F840F2FF11206836
:103F5000FDF746FA2168D1F8FC17814202D0022011
:103F600000F0BCF840F2FF311E48FDF739FA1D4958
:103F7000D1F8FC1F814206D020680079800702D466
:103F8000032000F0ABF81848007881074FF00100DB
:103F900001D5287070BD0F490870FEF75CFFBDE8C1
:103FA00070400120FFF7CFBD0A4910B5002008700E
:103FB000FEF751FF08480068007A800701D5FFF737
:103FC000FBFDBDE810400120FFF7BDBD300610002D
:103FD000B860000009031000E4021000FC021000A9
:103FE0000A0310004C000120303E012008B5FFF705
:103FF00039FD00F0B2F91B4C20680079800701D52B
:10400000FFF7B7FD20680079C00701D0FFF75BFF1D
:104010002168C87B00070DD511F86C0F497848431B
:1040200000F096FA104900231A4608700146C02095
:1040300000F035FAFEF70FFF01216B460022032046
:1040400001F028FB0098C007F6D0FFF7EFFE012132
:10405000032001F0FEFAFCF757FDEDE701210320F4
:1040600001F0C8BAE402100018410120304C2F4A78
:10407000C4E900210168A1604168E16081682161B3
:10408000C16861610169A1614169E1618169216280
:10409000C069606204F12800FDF74BFA01F013FCDF
:1040A000606400F035F82249224AC1E900207047D7
:1040B00010B501284FF0000205D00146BDE81040C0
:1040C000022000F002B90121022000F0FEF800F009
:1040D0001FF8012801D10220EAE7704710B5044615
:1040E00001460022032000F0F0F8012C01D0022C40
:1040F00001D100F00DF810BD00220146062000F0AD
:10410000E4B801460022072000F0DFF800F000F8D4
:10411000FCF743FB4FF0005010F8361F41F002014E
:104120000170817821F002018170FEE7AF0550FA3D
:1041300000EE0120BA0110AB77B585B00E46BDF890
:1041400014401546200A40EA0420ADF814004F48F8
:10415000BDF8141000240180A0F58070CDE90004A2
:104160004B480294039400681346484AC0790221E0
:10417000FCF737FC08B02A463046BDE87040454998
:1041800001F00FBC17B581B00B46BDF80400144612
:10419000010A41EA0020ADF804003C48BDF80410D3
:1041A00020F8021B194601F0FCFB00200090384863
:1041B0000023364A0068A11CC079FCF7E1FB1FBD53
:1041C00077B585B00E46BDF814401546200A40EA82
:1041D0000420ADF814002D48BDF81410002401800F
:1041E0002C48CDE900042A48029403940068134641
:1041F000264AC0790221FCF7F4FB08B02A46304673
:10420000BDE87040234901F0CCBBFCF7A9B908B563
:104210000020ADF8000002226946FFF78DFFBDF8CF
:10422000000008BD00B587B0002201210720FCF77F
:10423000BDFC072001F002FD00204FF4FA7100BF21
:10424000401C8842FBDB072001F001FDFFF7DFFF88
:10425000A0F584410E3902D00120FFF729FFAFF20B
:10426000DB000190AFF22F100090AFF2AB00029094
:10427000AFF2690003900848049040F28F20ADF837
:1042800014006846FCF732FD07B000BD184001205D
:10429000E4021000183F0120030500001CB5DB23D9
:1042A0008DF800308DF801008DF80210100E8DF899
:1042B0000300100C8DF80400100A8DF805008DF82D
:1042C0000620684600F032F91CBD1CB50F238DF89E
:1042D00000308DF801008DF80210080A8DF80300F7
:1042E0008DF80420100A8DF80500100C8DF80600DA
:1042F000100E95498DF80700012008706846FCF7FC
:1043000012FC1CBD2DE9FC41002706460097122037
:1043100015460C4601978DF800001AE0200A8DF82A
:104320000100C4F30B008DF80240315C30448DF87D
:10433000031041788DF8041081788DF80510C0784D
:104340008DF806008DF80770684600F0EFF8241D20
:104350002D1F002DE2DCBDE8FC811CB500207B494F
:1043600000900190096810234A7889788DF8003010
:104370008DF804008DF801008DF805208DF80200FD
:104380008DF806108DF803008DF80700684600F0E0
:10439000CDF81CBD70B588B00024009414200194A1
:1043A0008DF80000FDF7E6F88DF8010022208DF869
:1043B0000300664E66208DF804003068624D417837
:1043C0008DF8051080788DF80600287880018DF82A
:1043D0000700684600F0AAF80094152001948DF8B3
:1043E0000000306890F8EC178DF8011090F8ED1788
:1043F0008DF8021090F8EE178DF8031090F8EF0783
:104400008DF80400287880018DF80700684600F0D8
:104410008DF8009402A80194FCF7BDFF1B208DF8D5
:1044200000000298000E8DF801000298000C8DF833
:1044300002000298000A8DF8030002988DF804002B
:104440008DF8054004988DF80600287880018DF8D5
:104450000700684600F06AF800941C208DF8000000
:1044600003980194000E8DF801000398000C8DF85C
:1044700002000398000A8DF8030003988DF80400E9
:1044800005988DF8050006988DF8060028788001BB
:104490008DF80700684600F049F808B070BD1CB5FB
:1044A0002A4C246894F8E247A40710D5002401940C
:1044B000009416248DF800408DF801008DF802104C
:1044C0008DF803208DF80430684600F02FF81CBDED
:1044D0001CB5002300930193E1238DF800308DF883
:1044E0000100080A8DF80200100A8DF804008DF80A
:1044F00003108DF80520684600F018F81CBD1CB5A7
:10450000124A126892F89320D2070ED0002200922D
:104510000E2301928DF800308DF801008DF8061001
:104520008DF80720684600F001F81CBD10B5044660
:10453000012001F010F92046FCF7F5FABDE8104023
:10454000012001F023B90000C8021000E4021000AD
:10455000F0B52349074601200A68518C59B3214917
:10456000096891F8693092F83A108B4202D009B18B
:10457000FF2920D102F1340602F12404B51C0021E8
:104580004FF6FF7C383208E034F811300BB1634548
:1045900001D1002003E0491C89B2B942F4D331882B
:1045A00009B1FF2900D10020298821B1FF2902D0BB
:1045B0001288914200D20020F0BDF0B50024059E83
:1045C0000AE031F9145032F814705D4395FBF7F5A9
:1045D00020F81450641CA4B2B442F2DBF0BD000019
:1045E000E8021000E402100070B54A21304801F0E2
:1045F00057FA2F4CA6202F4D208042F26620608073
:1046000028684178217180786071FCF7AFFFE08005
:10461000FFF7FDFD2081286890F86C10217790F855
:104620006D1061772449E183244921842449618400
:104630002449A1872449A1842449E184244921856E
:10464000D0F8FC170A0C6285A185B0F83F10E1850F
:10465000B0F841102186B0F843106186B0F84510DB
:10466000A18690F8741001F0030284F83620C1F39B
:10467000011184F8371090F8681001F001012187CA
:10468000144909684A8952BA628701F12202E28715
:104690003232A4F8422090F8690004F8440F91F8EF
:1046A0003A0060700C4824F8020F0C48608070BD1E
:1046B00000000120E40210001A4101204E3E0120BA
:1046C000803E0120B23E012066410120C000012051
:1046D000303E0120E80210002C3E01202E3E012039
:1046E00010B5FBF793FEFCF702FF08B1FCF7F9FEEB
:1046F000BDE81040FBF788BE30B501230CE000EBAD
:10470000430531F8134025F8024C01EB430434F81B
:10471000024C20F813409B1C9342F0D330BD10B5DF
:10472000FBF774FEFCF7E3FE08B9FCF7D4FEBDE826
:104730001040FBF769BEF0B5851ADDE905471E1B81
:1047400075438E1A012F02D0904206DD0BE0904295
:1047500001DC1846F0BD884201DB2046F0BD95FB28
:10476000F6F0181AF0BD8842F3DA95FBF6F0204413
:10477000F0BD2DE9FC4F04468F480B460026076824
:10478000354607F58A7207F58E7C125707F5927841
:1047900007F5967107F59A7907F59E7A07F5A27BDA
:1047A000184607F5A6779A4200DD10460957994248
:1047B00000DA084682420ADC1CF90430834206DB38
:1047C000194619F9043001251AF9044008E018F9CE
:1047D0000420824209DC814207DB3B571BF904407D
:1047E000CDE90045FFF7A7FF46B23046BDE8FC8F94
:1047F0002DE9F84F894670490546DFF8C0A10868E1
:104800009B46904690F8E307882808D12A68CAF8A2
:1048100000206A68CAF80420AA68CAF808200024A0
:104820005AE0674839F81410634B076838F81400E9
:104830000126081A25F814001868243790F8E317A1
:10484000882906D139F8142038F81410511A2AF89A
:104850001410C07BC0063DD55A480078D0BB5A48DA
:104860000078012836D15948007898B3A0B259464B
:10487000FFF77FFF01465048006890F8E30788285B
:1048800005D1534880F830B2204480F831120AEB49
:1048900044008181F1B135F9140064225043C1F123
:1048A000640290FBF2F000B2002802DA00264042D7
:1048B00000B237F81420824205DC821A4A43642190
:1048C00092FBF1F1401A25F814001EB980B2404263
:1048D00025F81400641C24B20A988442A1DB3648EF
:1048E000006890F8E307882835D12968CAF81810BD
:1048F0006968CAF81C10A968CAF820100620009040
:104900002F482E490268183101F10C00938E243291
:10491000FFF753FE2E4F2F4E6FF0130530883D5496
:10492000401C30800024A0B22946FFF722FF3188C6
:10493000641C24B27854491C3180062CF3DB6D1CB6
:104940006DB23C2DEADB3088B0F50C7F07F800B083
:1049500001D300203080BDE8F88F70B5002408E056
:1049600031F8145032F81460AD1B20F81450641C58
:1049700024B29C42F4DB70BDF0B4049C012C04D042
:104980001BB1C3F11006002412E0F0BC520001F08C
:1049900008B830F9145031F914705D4307FB06551F
:1049A000EF1705EB17752D1120F81450641C24B275
:1049B0009442EEDBF0BC7047E4021000D0430120CB
:1049C000E8021000EC021000184101200903100059
:1049D00098410120CA0210000FB42DE9F05F0025B4
:1049E000DDF874A08B4681462E464FF0010808FA88
:1049F00006F7002407EA0B076FB108FA04F010EA83
:104A0000090F08D0324621460C9800F0CFFA0AF878
:104A100005006D1CEDB2641CE4B2052CECD3761CD1
:104A2000F6B2052EE3D3BDE8F01F5DF814FB10B518
:104A3000044650212B4801F033F82B4A1178491CC9
:104A40001170A00504D5BDE81040264800F001B85B
:104A500010BD2DE9F041044690B0A52020704FF420
:104A60000070A4F8010000F0A8F9207100F0A0F98E
:104A7000607100F098F9804600F090F905461B48F7
:104A800000680179552904D1D0F8050020F07F4055
:104A9000A060174E392206F1740796F8B000207313
:104AA00004F130000F90391D684600F0BFFF00226E
:104AB00029464046736FFFF78FFF04F110000F90F7
:104AC0003922391D684600F0B1FF012229464046CF
:104AD000736FFFF781FF04480078E07010B0BDE805
:104AE000F081000000800120CC021000E8021000DC
:104AF0004C00012070B5854E05460C46306890F894
:104B0000940001070AD5E10700F007004FF000020A
:104B100001D0012100E00021FCF748F8306890F84E
:104B2000941008060AD5A007C1F302104FF0000246
:104B300001D5012100E00021FCF738F8306890F839
:104B4000950001070AD5690700F007004FF0000241
:104B500001D5012100E00021FCF728F8306890F829
:104B60009610080712D56A48007878B1694800782D
:104B700060B96948007848B96848007800284FEA69
:104B8000847008D0002810D1A8070ED101F00700CA
:104B90000022114605E00028F6D001F007000022AF
:104BA0000121BDE87040FCF701B870BD10B5574C4D
:104BB000206890F8940001071CD500F0070001F070
:104BC00046F8206890F8940000F0070001F036F8ED
:104BD00020680022114690F8940000F00700FBF7CF
:104BE000E5FF20680022114690F8940000F00700CD
:104BF000FBF7F2FF206890F8940001061CD5C0F383
:104C0000021001F024F8206890F89400C0F302101C
:104C100001F014F820680022114690F89400C0F3C7
:104C20000210FBF7C3FF20680022114690F89400A1
:104C3000C0F30210FBF7D0FF206890F89500010741
:104C40001CD500F0070001F002F8206890F89500EC
:104C500000F0070000F0F2FF20680022114690F8F3
:104C6000950000F00700FBF7A1FF20680022114625
:104C700090F8950000F00700FBF7AEFF206890F871
:104C8000950001061CD5C0F3021000F0E0FF20687B
:104C900090F89500C0F3021000F0D0FF20680022C9
:104CA000114690F89500C0F30210FBF77FFF2068D3
:104CB0000022114690F89500C0F30210FBF78CFF1C
:104CC000206890F8960001071ED500F0070000F05C
:104CD000BEFF206890F8960000F0070000F0AEFFDD
:104CE00020680022114690F8960000F00700FBF7BC
:104CF0005DFF20680022114690F89600BDE8104044
:104D000000F00700FBF768BF10BD0000E4021000D0
:104D100009031000EC021000ED02100094021000D4
:104D200010B500F001F91B490020086010BD10B556
:104D3000FFF7B9F9BDE81040FBF7CBBE00210160D9
:104D40004160704710B5017999B1134900220A609A
:104D50004A608A60CA600F49D0E90020C1E9012099
:104D6000081D00F01FF90B48001D00F0B3F90120E9
:104D700010BD002010BD10B50749064C0870206812
:104D80008860201D0168044888472068401C206016
:104D900010BD0000D002100050061000FD48006851
:104DA00090F86A007047FB48006890F86B00704705
:104DB000F848006890F86C007047F648006890F872
:104DC0006D00704770B5040004D1FBF782FFF34912
:104DD000F1484860F248F34A002101701160F2483E
:104DE00001230360450685F8EE10F04EA0253560DE
:104DF000016013602046BDE87040FFF7BCBF10B5EE
:104E00000446142100F06EFE0020207080206070A7
:104E1000A020A070FFF7C7FFE070FFF7BFFF207171
:104E2000FFF7C6FF6071FFF7C8FFA071D948E279AC
:104E3000006810F8771F61F38612E27110F8051907
:104E4000490861F3C712E271C18821818168E1607C
:104E50000378217C63F30001217403785B0863F31A
:104E60004101217403789B0863F382012174037864
:104E7000DB0863F3C301217403781B0963F3041196
:104E8000217403785B0963F34511217403789B094E
:104E900063F3871121744378617C63F300016174CB
:104EA00043785B0863F34101617443789B0863F3C3
:104EB000820161744378DB0863F3C3016174437852
:104EC0001B0963F30411617443785B0963F34511B3
:104ED000617443789B0963F386116174837863F38B
:104EE0000102E27183789B0863F38202E2718378A6
:104EF0001B0963F3C402E27183789B0963F34512D3
:104F0000E271C27862F3C7116174C1780A09A17CA9
:104F100062F30101A174007960F38201A17420465B
:104F2000BDE81040FBF777BF2DE9F0419C48002415
:104F30004FF0E027047044708470C47004714FF027
:104F400080764FF00108C7F880619948A02580F865
:104F50000054202297499848843700F067FD934811
:104F600008380560954804608F49091DC1F8008024
:104F7000710181F8DE80C7F8FC61FE673D2290492F
:104F8000A020FCF78BF88E48743890F8B000FCF73E
:104F90008AF88C48FFF733FFBDE8F04189481430A8
:104FA00000F0D4B87E49002008707047844B02EBB3
:104FB0004202743B03EB820202EB410110B191F813
:104FC0007500704791F8740070472DE9F041DFF8E3
:104FD000C4C102460024714D0127714BDCF800006A
:104FE000052912D0042949D0FFF7DDFED070FFF764
:104FF000D5FE1071FFF7DCFE5071FFF7DEFE9071F9
:10500000BDE8F0411046FBF776BE017A490726D588
:1050100093F903100CE090F86E6007FA01FE16EAAF
:105020000E0F04D0D9701979491C197102E0491C7E
:105030000529F0DBD97890F86A6007FA01FE06EAE4
:105040000E061671577193F904606E73491CD9707E
:1050500090F86C10B14209DCDC701C7106E06C73D6
:1050600090F86E10117190F87010517190F86F00F7
:10507000D070DCF8000090F87100C0E793F90110DF
:105080000CE090F86A6007FA01FE16EA0E0F04D0F1
:1050900059709978491C997002E0491C0529F0DB88
:1050A0005771597810F86A6F8F403E4016714078FA
:1050B000D070DCF80000491C90F86D60967193F98F
:1050C00002602E73597090F86C00B04298DC5C70EE
:1050D0009C7095E730B5047989B0B4B12021684659
:1050E00000F000FD6D4621463648FFF76EFF35495A
:1050F00020221431284600F099FC0025062C10D2FD
:10510000DFE804F00F0F060D060609B0012030BDE0
:105110002048006890F890008DF8110001E08DF8AB
:105120001F506846FBF791FE1D49012008701F487B
:105130000C3805601120410781F8EE00E5E71848BA
:105140000078012801D1FBF7B4BD7047AFF28B3175
:105150000160114981603231C160002101740D4943
:10516000096811F8802F42744A7882744A888282D2
:105170008A88C282CA8802830A8942834A898283D2
:105180000A7B8277497B01F01F01C17741F28831A8
:1051900081807047E40210001A410120500610007F
:1051A000DC02100010050022901B0022100C0220CF
:1051B00018E000E07861000000000220E01E0022FC
:1051C000C00001206006100010B5FCF7A8F9FBF73D
:1051D000D7FABDE81040FFF7A2BA0AF15BBD10B5DF
:1051E000FFF7F2FF10BD10B5FFF7EEFF10BD10B5D1
:1051F000FFF7EAFF10BD10B5FFF7E6FFBDE810406E
:10520000FEF72CBF10B5FFF7DFFF10BD10B5FFF79D
:10521000DBFFBDE81040FBF7B9B910B5FFF7D4FFCD
:10522000BDE81040FBF7F0B910B5FFF7CDFFBDE8C2
:105230001040FBF712BA10B5FFF7C6FF10BD10B54E
:10524000FFF7C2FFBDE81040FBF72FBA10B5FFF71C
:10525000BBFFBDE81040FBF76EBA10B5FFF7B4FF17
:1052600010BD10B5FFF7B0FF10BD10B5FFF7ACFFD4
:1052700010BD10B5FFF7A8FF10BD10B5FFF7A4FFD4
:1052800010BD10B5FFF7A0FF10BD10B5FFF79CFFD4
:1052900010BD10B5FFF798FF10BD7047704710B5EF
:1052A000FFF792FFBDE81040FBF7A7BA70477047C1
:1052B0007047704710B5FFF787FFBDE81040FFF754
:1052C0003EBF704730B58DB042F26620FCF72DF935
:1052D000FCF7E9F84FF400624B494C4800F0A6FB9C
:1052E0004FF480524A494B4800F0A0FBFBF7D2FB39
:1052F0000120FBF7E6FBFBF77BFF0E246846FBF77C
:1053000099FF0698C01C65D00698401C64D006988A
:10531000801C61D00698C4B22046FCF7F3F8FCF775
:10532000DAF8FCF72BF93C4C20680078A52802D06D
:105330000120FEF7D3FE40F2FF112068FCF750F881
:105340002168D1F8FC17814202D00220FEF7C6FE88
:1053500040F2FF312F48FCF743F82E49D1F8FC1FEB
:10536000814206D020680079800702D40320FEF72E
:10537000B5FEFBF7F9FBFBF74BF82948274D016811
:10538000087955282CD07020FEF7B6FE2846FBF78A
:10539000C8F8FBF7BBFA20680079400704D421491C
:1053A00000200860091F0860FEF73CFFFFF7B8FC0B
:1053B000FBF7F8F938B1002211460120FEF785FF0E
:1053C0000120FEF770FEFBF7D6F90DB0BDE83040C6
:1053D000FFF7ECBB312000E03020FEF78DFE9BE7AD
:1053E000D1F8050020F07F45D0E710B5FBF70EF8A7
:1053F000FFF768FFFFF7F8F800F016F8FBF704F87E
:1054000000F07EF8012010BDF0EF030000F0012055
:10541000F0CF03004C000120E402100000770100EF
:10542000E8021000841400227FB500F041F81F4DFF
:10543000002405EB441000F11002017F4CCACDE9B5
:105440000261CDE900230FC800F0DAF910B10220A3
:10545000FEF757FE641C052CEBDB144D0024A03531
:1054600004EB440005EB800155F820008A68496888
:1054700000F046F910B10220FEF743FE641C042C34
:10548000EEDB0A4D0024D03505EBC400416855F829
:10549000340000F08FF810B10220FEF732FE641CD9
:1054A000042CF1DB7FBD0320FEF72BBE98610000CA
:1054B0001A4910B5012008701949002008601949DF
:1054C0000860194908601949086000F07DF900F08A
:1054D0000FF900F067F8002010BD10B5124800F079
:1054E00024FA104908600E490968884207D00B4821
:1054F0000078022803D1BDE81040FAF73FBF10BD85
:1055000010B5FFF7EAFF054902200870FAF71AFF05
:105510004FF0FF3010BD0520704700000B03100056
:105520000C031000100310001403100018031000E7
:1055300070B50D460446C1698068CC2200F0A8FA17
:10554000E169A068084440384FF08071C163216A66
:105550008163002141630163C1628162C0E9085136
:105560004FF00B31C1614FF00A3181614FF00931C9
:1055700041614FF0083101614FF00731C1604FF0D8
:10558000063181604FF0053141604FF00431016018
:1055900070BD82698168914202D84068FFF783BF7D
:1055A0007047000010B54FF4B4714F4800F09AFAFC
:1055B000002010BD70B5054600EBC5014A4800EB60
:1055C0008104FAF713FF0646207828B13046FAF72F
:1055D00015FF6FF0010070BD032020700020656092
:1055E000206204F11C0000F079F93046FAF706FF5A
:1055F000002070BD2DE9F0410F463B49002500EB2E
:10560000C00001EB80042E46FAF7F0FE8046206AC7
:105610003843206204F11C00074600F086F90CE0D4
:10562000216A026C114203D000F026F9012600E045
:105630006D1C2946384600F06EF90028F0D1012E85
:1056400001D1FFF74AFF4046FAF7D8FE0020BDE837
:10565000F08170B50D46244900EBC00001EB8004D9
:10566000FAF7C4FE216AA9432162FAF7C7FE0020B7
:1056700070BD70B50C461C4900EBC00001EB800505
:1056800000202060FAF7B2FE296A2160FAF7B6FE20
:10569000002070BD2DE9F0410D46134900EBC0001C
:1056A0001E46904601EB8004FAF7A0FE07460F481D
:1056B00000680564216A294203D104F11C0100F04D
:1056C000EDF83846FAF79AFEFAF790FE216A29407B
:1056D0003160B8F1010F02D1216AA9432162FAF7C2
:1056E0008DFE0020B3E700009C1A10000C03100090
:1056F00010B54FF4C871324800F0F4F9002010BD25
:105700002DE9F041884605462D4900EB85001746F6
:1057100001EBC004FAF76AFE0646207830B1304645
:10572000FAF76CFE6FF00100BDE8F08102202070F6
:10573000E7611422414604F10800656000F031F988
:105740000020206204F1240000F0C8F83046FAF787
:1057500055FE0020E8E770B5194900EB800001EB29
:10576000C004FAF743FE0546D4E90701814205DB90
:10577000144804F12401006800F090F8206A401CED
:1057800020622846FAF73AFE002070BD70B50C4939
:1057900000EB800001EBC004FAF728FE0546206A02
:1057A00008B1401E206204F1240000F0BEF810B1E0
:1057B000606A00F011F82846FAF720FE002070BD5C
:1057C000041C10000C03100010B54FF42A7140485F
:1057D00000F088F9002010BD10B5044690F838009C
:1057E00002280BD0204600F0A2F8022084F83800EE
:1057F0003849204600F076F8FFF76FFE002010BD14
:105800002DE9F05F8B460646314900EB06109046C5
:10581000DDE90AA911F820201D461AB16FF0010038
:10582000BDE8F09F01EB8004FAF7E0FD0746012098
:105830002070C4E90165C4E90585C4E907A91422FB
:10584000594604F1240000F0ACF8002084F8370039
:1058500084F838006169E0602061C4E90F102046D7
:105860000C99FFF765FEA0602046FFF7B5FF3846AC
:10587000FAF7C4FD0020D3E710B5044690F83800CD
:10588000022809D0204600F052F8022084F838009F
:105890001049204600F026F8002010BD70B50446DF
:1058A00090F838000D4602280BD1204600F03FF852
:1058B000032084F838002946204600F013F8FFF74B
:1058C0000CFE002070BD044800684068704700006E
:1058D000941D1000140310000C031000002101603F
:1058E0000846704730B50A6812B10B46C46B09E030
:1058F00000220860C0E903210BE000BF02F10C03A5
:10590000D26812B1D56BA542F8DC1A68C0E9032150
:105910001860002030BD0068002201E0C068521C01
:105920008A4201D00028F9D17047006870470269A7
:105930000AB1116831B96FF00400704701F10C022F
:10594000C96839B18142F9D1C9681160002101618A
:10595000084670476FF00300704710B54C1084EA9A
:10596000530404D54042C1F1000138BF491E1B4217
:1059700004D55242C3F1000338BF5B1E00F0D9F8D2
:1059800014F0804F04D04042C1F1000138BF491EDD
:1059900014F0004F04D05242C3F1000338BF5B1E25
:1059A00010BD032A40F2308010F0030C00F0158087
:1059B00011F8013BBCF1020F624498BF11F801CB12
:1059C00000F8013B38BF11F8013BA2F1040298BF77
:1059D00000F801CB38BF00F8013B11F0030300F0E1
:1059E0002580083AC0F0088051F8043B083A51F885
:1059F00004CBA0E80810F5E7121D5CBF51F8043B8A
:105A000040F8043BAFF30080D20724BF11F8013BFC
:105A100011F801CB48BF11F8012B24BF00F8013B5E
:105A200000F801CB48BF00F8012B704710B5203AB1
:105A3000C0F00B80B1E81850203AA0E81850B1E847
:105A40001850A0E81850BFF4F5AF5FEA027C24BFFD
:105A5000B1E81850A0E8185044BF18C918C0BDE8F4
:105A600010405FEA827C24BF51F8043B40F8043BBD
:105A700008BF7047D20728BF31F8023B48BF11F872
:105A8000012B28BF20F8023B48BF00F8012B7047CC
:105A900002F0FF0343EA032242EA024200F002B8A6
:105AA0004FF000020429C0F0128010F0030C00F047
:105AB0001B80CCF1040CBCF1020F18BF00F8012BC5
:105AC000A8BF20F8022BA1EB0C0100F00DB85FEA93
:105AD000C17C24BF00F8012B00F8012B48BF00F85F
:105AE000012B70474FF0000200B5134694469646CE
:105AF000203922BFA0E80C50A0E80C50B1F12001E1
:105B0000BFF4F7AF090728BFA0E80C5048BF0CC08E
:105B10005DF804EB890028BF40F8042B08BF7047EC
:105B200048BF20F8022B11F0804F18BF00F8012B5E
:105B3000704753EA020C00F069802DE9F04B4FF0FA
:105B40000006002B1FBFB3FA83F503FA05F424FA0D
:105B500005F65E4012BF1643B2FA82F502FA05F46A
:105B6000C5F120051EBF22FA05FC44EA0C042035CD
:105B700056EA044C4FEA144418BF641C4FF0000866
:105B80004FF00009904271EB030C39D3002919BF83
:105B9000B1FA81F701FA07F6B0FA80F700FA07F6D2
:105BA000C7F120071EBF20FA07FC46EA0C06203783
:105BB000B6FBF4FCA7EB0507103F07F01F0BCBF17A
:105BC00020060CFA0BFB2CFA06F644BFB34600265F
:105BD000202FA4BF5E464FF0000B5BEA060C08BF07
:105BE0004FF0010B19EB0B09ABFB027C48EB0608ED
:105BF000C01B06FB02CC0BFB03CC71EB0C01C1E715
:105C00000B46024641464846BDE8F08B13B54FF0BF
:105C100000004FF00001AFF30080BDE81C4070476A
:105C20000446AFF300802046FAF7CAFA7047000036
:105C300001491820ABBEFEE7260002000121814089
:105C40004FF0005010F8352F8A4302707047012141
:105C500081404FF0005010F8352F0A430270704712
:105C600010B50B480A4A007851789278012803D879
:105C7000012901D8012A09D9064B1B6893F8E3379B
:105C8000FA2B01D1FEF70AFB012010BD002010BD48
:105C90008B021000E4021000441D0A5D3F1E1D1D12
:105CA00006080708220F052F200F0F0F0204040417
:105CB0001108031810080808000202020904020C67
:105CC00008040404000101015A280D7B54282828E7
:105CD000090B090B2D14073E2A141414040605069B
:105CE000170A041F150A0A0A010303030C05021010
:105CF0000B05050500020202000101020102020378
:105D00000102020302030304000000001B000080E4
:105D10002D00008036000000410000805A00000085
:105D20006C00000077000080990000808200000075
:105D3000B4000000AF000080D8000000C300008065
:105D4000F5000080EE000000290100803201000013
:105D5000040100001F010080680100007301008041
:105D6000450100805E010000B0010000AB01008031
:105D70009D01008086010000F1010080EA01000021
:105D8000DC010000C70100804902008052020000CF
:105D9000640200007F0200800802000013020080FD
:105DA000250200803E020000D0020000CB020080ED
:105DB000FD020080E6020000910200808A020000DD
:105DC000BC020000A7020080600300007B0300808B
:105DD0004D03008056030000210300803A030000B9
:105DE0000C03000017030080F9030080E2030000A9
:105DF000D4030000CF030080B8030000A303008099
:105E0000950300808E030000890400809204000046
:105E1000A4040000BF040080C8040000D304008074
:105E2000E5040080FE040000100400000B04008064
:105E30003D04008026040000510400804A04000054
:105E40007C04000067040080A0050000BB05008002
:105E50008D05008096050000E1050080FA05000030
:105E6000CC050000D7050080390500802205000020
:105E7000140500000F050080780500006305008010
:105E8000550500804E050000C0060000DB060080BE
:105E9000ED060080F6060000810600809A060000EC
:105EA000AC060000B70600805906008042060000DC
:105EB000740600006F0600801806000003060080CC
:105EC000350600802E060000E9070080F20700007A
:105ED000C4070000DF070080A8070000B3070080A8
:105EE000850700809E070000700700006B07008098
:105EF0005D07008046070000310700802A07000088
:105F00001C07000007070080090900801209000033
:105F1000240900003F09008048090000530900805F
:105F2000650900807E090000900900008B0900804F
:105F3000BD090080A6090000D1090080CA0900003F
:105F4000FC090000E7090080200800003B080080F1
:105F50000D08008016080000610800807A08000023
:105F60004C08000057080080B9080080A208000013
:105F7000940800008F080080F8080000E308008003
:105F8000D5080080CE080000400B00005B0B0080AD
:105F90006D0B0080760B0000010B00801A0B0000D7
:105FA0002C0B0000370B0080D90B0080C20B0000C7
:105FB000F40B0000EF0B0080980B0000830B0080B7
:105FC000B50B0080AE0B0000690A0080720A000069
:105FD000440A00005F0A0080280A0000330A00809B
:105FE000050A00801E0A0000F00A0000EB0A00808B
:105FF000DD0A0080C60A0000B10A0080AA0A00007B
:106000009C0A0000870A0080800D00009B0D008024
:10601000AD0D0080B60D0000C10D0080DA0D00004E
:10602000EC0D0000F70D0080190D0080020D00003E
:10603000340D00002F0D0080580D0000430D00802E
:10604000750D00806E0D0000A90C0080B20C0000E0
:10605000840C00009F0C0080E80C0000F30C008012
:10606000C50C0080DE0C0000300C00002B0C008002
:106070001D0C0080060C0000710C00806A0C0000F2
:106080005C0C0000470C0080C90F0080D20F00009C
:10609000E40F0000FF0F0080880F0000930F0080C6
:1060A000A50F0080BE0F0000500F00004B0F0080B6
:1060B0007D0F0080660F0000110F00800A0F0000A6
:1060C0003C0F0000270F0080E00E0000FB0E008058
:1060D000CD0E0080D60E0000A10E0080BA0E00008A
:1060E0008C0E0000970E0080790E0080620E00007A
:1060F000540E00004F0E0080380E0000230E00806A
:10610000150E00800E0E0000D33B00000F3C000077
:106110007D3E0000773E0000253A0000253A000051
:10612000253A00004D3B0000253A0000313D0000BB
:10613000233C0000D13C0000533C0000AF3C000079
:10614000973E0000D13E0000EF3A0000F33A000015
:10615000833E0000673D0000253A0000233B00001D
:10616000253A0000BF3B0000C93B0000253A000073
:10617000933E0000253A0000E33E0000593F000036
:10618000713B0000A73B0000253A0000253A0000C3
:10619000253A0000253A0000253A0000253A000083
:1061A000253A0000253A0000253A0000253A000073
:1061B000253A0000253A0000253A0000253A000063
:1061C000253A0000253A0000046C00080000047C19
:1061D00003430001187801001A604002400C0300DC
:1061E0000782000C0D000000000000008862000023
:1061F00005000000DC06100000040000151B000074
:10620000000000000200000001000000DC6200004D
:1062100004000000DC0A100040060000B12200006B
:106220000000000002000000020000000C630000FB
:10623000030000001C11100000080000F1380000ED
:10624000000000000200000003000000A86200003F
:10625000020000001C191000000100009D3F00001A
:10626000000000000200000004000000B86200000E
:10627000010000001C1A100080000000E939000035
:10628000000000000200000000000000B0620000FA
:106290000100000001000000E862000001000000B1
:1062A00002000000F4620000010000000300000092
:1062B000C4620000010000000000000094620000C1
:1062C00001000000D0620000020000000463000032
:1062D00003000000A062000054736B5F53537663A9
:1062E00000000000456C665F537376630000000099
:1062F000456C665F436D640054736B5F436D64006F
:1063000053656D5F4166650054736B5F49646C65EE
:106310000000000053656D5F4D54427566660000D5
:10632000456C665F5363616E0000000054736B5FE1
:106330005363616E0000000053656D5F45767446DF
:1063400069666F0053656D5F43616C696246726197
:106350006D657300456C665F4D74000054736B5F30
:106360004D74000044630000000210001C01000096
:106370001C0100006064000000FC1000040100002B
:106380001C010000606400001C031000201D0000C0
:1063900038010000000000000000000000000000C4
:1063A00000000000000000000000000000000000ED
:1063B00000000000000000000000000000000000DD
:1063C00000000000000000000000000000000000CD
:1063D00000000000000000000000000000000000BD
:1063E00000000000000000000000000000000000AD
:1063F000000000000000000000000000000000009D
:10640000000000000000000000000000000000008C
:10641000000000000000000000000000000000007C
:10642000000000000000000000000000000000006C
:10643000000000000000000000000000000000005C
:10644000000000000000000000000000000000004C
:10645000000000000000000000000000000000003C
:10646000000000000000000000000000000000002C
:10647000000000000000000000F001204C0001209E
:10648000000000000000000000000000000000000C
:1064900000000000000000000000000000000000FC
:1064A00000000000000000000000000000000000EC
:1064B00030B572B601250D4C256000236A0701290D
:1064C00010D082F86B3000F03F0082F86A00084874
:1064D000056001680029FCD105481C300360236079
:1064E00062B630BD402182F86B10ECE7401B002201
:1064F0005C0D0022FCB54FF00052D02082F8C300A2
:106500002B4F386848B140F29B70D0844520A2F8E8
:106510005200A2F85200FA2008E040F22F30D08456
:106520003120A2F85200A2F85200BC20402482F888
:106530002040442582F8205000234FF49676CDE980
:106540000063194605E00099491E00910199491C14
:1065500001918142F7D30FE082F8204082F8205069
:10656000CDE90063194605E00099491E00910199A3
:10657000491C01918142F7D392F82010C906EBD44F
:1065800082F8C330386828B141F29840D08440F294
:10659000572004E041F22C00D08440F2C110A2F850
:1065A0005200A2F852004C2082F82000FCBD0000EE
:1065B000DC040022A51000000100004A0705194D67
:1065C00001FF961F0C100F23DC052C01DC052C01AC
:1065D00000000000D00700000000000000000709D4
:1065E0003200000000000000000000000000070171
:1065F0000A05005E015E01FA000000966464005E18
:1066000001E8039600940214053408E40C6E0F00B0
:1066100000000000200300910032000000011A0574
:1066200003021A0401013F0244000003000100803C
:10663000000000001E01400696000800E50064000E
:106640001F04000010000001980A0B640000000005
:1066500000000000030010051014000000000000FE
:10666000000000005300024B03320064283C401F2E
:10667000701732A00FB80BA00FB80B2D0164643255
:1066800064003200003C000045960000050C00004C
:106690000301000006090000408000408000000067
:1066A00000000000000000000000000000000000EA
:1066B00000000000000000000000000000000000DA
:1066C0000000000000000000ECECECECECEC000042
:1066D00000000000000000002D2D2D2D2D2D0000AC
:1066E0003C3C3C3C3C3C0000323232321919000048
:1066F0000F031F0305060000141E141B191E0000C3
:10670000323A4537323D00000000102788137017D9
:106710007017B80B100EB036B036B036401F401FA1
:10672000401FAC0DE803A00F2003C8002003960013
:1067300032003200000000000000000000000000F5
:106740000000000000000000000000000000000049
:106750000000000000000000000000000000000039
:106760000000000000000000000000000000000029
:106770000000000000000000000000000000000019
:106D900000000000000002000000000000000000F1
:106DA0000F000000000000000000000000000000D4
:086DB0002DFF039F37F9C66FA8
:00000001FF
